:020000040800F2
:1000000000040120010200080302000803020008A6
:1000100003020008030200080302000803020008AC
:10002000030200080302000803020008E12F000891
:10003000030200080302000803020008030200088C
:10004000030200080302000803020008030200087C
:1000500003020008030200083D320008693200086C
:1000600095320008C1320008ED3200080302000892
:10007000030200080302000803020008030200084C
:10008000030200080302000803020008030200083C
:1000900003020008030200080302000819330008E5
:1000A000030200080302000803020008030200081C
:1000B0006130000803020008030200080302000880
:1000C00003020008030200080302000803020008FC
:1000D00003020008030200080302000803020008EC
:1000E000813300080302000803020008030200082D
:1000F00003020008030200080302000803020008CC
:1001000003020008030200080302000803020008BB
:1001100003020008030200080302000803020008AB
:10012000030200080302000803020008030200089B
:10013000030200080302000803020008030200088B
:10014000030200080302000803020008E126000879
:10015000030200080302000803020008030200086B
:10016000030200080302000803020008030200085B
:10017000030200080302000803020008030200084B
:10018000030200080302000803020008030200083B
:10019000030200080302000803020008030200082B
:1001A000030200080302000803020008030200081B
:1001B000030200080302000803020008030200080B
:1001C00003020008030200080302000803020008FB
:1001D00003020008030200080302000803020008EB
:1001E00003020008030200080302000803020008DB
:1001F00003020008030200080302000803020008CB
:1002000002E000F000F8FEE772B6394880F3088893
:10021000384880F3098838484EF60851CEF200017C
:10022000086040F20000CCF200004EF63471CEF2CD
:1002300000010860BFF34F8FBFF36F8F40F20000E3
:10024000C0F2F0004EF68851CEF200010860BFF314
:100250004F8FBFF36F8F4FF00000E1EE100A4EF6A4
:100260003C71CEF200010860062080F31488BFF3D1
:100270006F8F01F0B9FE02F03BFE4FF055301F4981
:100280001B4A91423CBF41F8040BFAE71C49194A4A
:1002900091423CBF41F8040BFAE71A491A4A1B4B3A
:1002A0009A423EBF51F8040B42F8040BF8E70020D5
:1002B0001749184A91423CBF41F8040BFAE701F094
:1002C000D7FE02F07FFE144C144DAC4203DA54F812
:1002D000041B8847F9E700F03FF8114C114DAC4280
:1002E00003DA54F8041B8847F9E701F0BFBE0000A9
:1002F000000401200024012000000008000001206B
:1003000000040120A037000800240120502401200F
:100310005024012068340120000200080002000877
:1003200000020008000200082DE9F04F2DED108AB0
:10033000C1F80CD0D0F80CD0BDEC108ABDE8F08F1D
:10034000002383F311882846A047002001F0F0FA2B
:1003500001F09CFA00DFFEE71B4B7B2270B51A70A0
:100360006FF07F0200245A720E225C709C70DC7069
:100370001C715C719C71DC711C729A72DC7201F0F0
:1003800009FE064601F02AFE054650B90F4B9E4273
:1003900017D001339E4241F2883412BF0546002433
:1003A0000125002001F0FCFD0DB100F0B7F800F0D0
:1003B00053FD00F04BFC204600F052F900F0AEF87F
:1003C000F9E70446EDE700BF50240120010007B023
:1003D00008B500F0DDFBA0F120035842584108BDEC
:1003E00007B5054B02211B88ADF8043001A800F0C9
:1003F0001DFC03B05DF804FB7C340008064991F84D
:10040000243033B100230822086A81F8243000F038
:1004100041BC0120704700BF702401202DE9F84F36
:10042000234C94F824300546884617468BBB2E464D
:10043000DFF87C90002F38D094F824A0BAF1000F98
:1004400005D12022FF214846266200F0F3FCCAF1C4
:100450000805BD4228BF3D465FFA85FBAD00414619
:100460002A4604EB8A0000F0BBFC94F82430A7EB8A
:100470000B079B445FFA8BFBBBF1080F2E44A8448B
:10048000FFB284F824B0D5D1FFF7B8FF0028D1D14E
:1004900008E0266A06EB8306B042C9D0FFF7AEFF3C
:1004A0000028C4D10020BDE8F88F0120BDE8F88FF6
:1004B0007024012010B572B6202383F3118862B630
:1004C0001248C3680BB101F0BBFA0023104A0F4871
:1004D0004FF47A7101F078FA002383F311880D4C00
:1004E000236813B12368013B2360636813B1636819
:1004F000013B6360084B1B7833B9636823B9022062
:1005000000F064FC3223636010BD00BF5C24012056
:10051000B5040008A0290120982401202DE9F0410C
:10052000454B464953F8042F013201D1BDE8F08113
:100530008B42F7D1424C434B22689A427AD9424BC4
:100540009B6803F1006303F5C0339A4272D2002026
:1005500000F098FB3D4B0220187000F02FFC3C4B44
:100560001A6C00221A64196E1A66196E596C5A6454
:10057000596E5A66596E596941F08001596159693D
:1005800021F0800159615969196941F000511961DF
:10059000196921F0005119611B6972B62D492E4B62
:1005A0000B601D682468BFF34F8FBFF36F8F2B4B19
:1005B000C3F88420BFF34F8F5A6922F480325A6106
:1005C000BFF34F8FD3F88020C2F3C906C2F34E3277
:1005D0005201B70743F6E07E02EA0E08384631467C
:1005E000013948EA000CB1F1FF3FC3F874C200F1D1
:1005F0004040F5D1203A12F1200FEDD1BFF34F8FDB
:10060000BFF36F8FBFF34F8FBFF36F8F5A6922F421
:1006100000325A610022C3F85022BFF34F8FBFF35C
:100620006F8F72B6202383F3118862B6AD4685F3CF
:1006300008882047BDE8F081FC7F01081C80010884
:1006400004800108FF7F0108502401209824012024
:100650000038024008ED00E00080010800ED00E0F5
:100660002DE9F04FB14C97B020228146FF210EA812
:10067000A66800F0DFFBAE4A1378A346B3B9AD48D5
:1006800001211170C36072B6202383F3118862B612
:10069000C3680BB101F0D4F90023A74AA5484FF471
:1006A0007A7101F091F9002383F31188B9F1000FF9
:1006B00002D0A24BC3F80090A14BA04A00241C70AA
:1006C0005460254627469846012000F077FBB9F193
:1006D000000F00F02282994B1B68002B40F01D8216
:1006E00017B0BDE8F08F0220FFF772FE002840F03F
:1006F0000E82944B1B88ADF82430022109A800F02B
:1007000095FAE1E74FF47A7000F042FA031E019384
:10071000EFDB0220FFF75CFE82460028E9D0019B58
:10072000581E042800F2F581DFE800F0030D1013D5
:10073000160016A8052340F8343D042100F076FA8F
:100740005446002752E004217848F7E704217E4808
:10075000F4E704217D48F1E71C24204600F094FAD8
:1007600004340990042109A800F060FA2C2CF4D17B
:10077000E6E7002DBDD0002CBBD00220FFF728FEFD
:100780000546002800F0C781012000F07BFA022016
:1007900088F8000000F012FB0024E3B21846019331
:1007A00000F080FA824648B1019B184600F08AFAB0
:1007B00001340028F1D12C46654B9BE70123022030
:1007C00088F8003000F0F0FA5646DBF808309E4218
:1007D00006D2304600F058FA0130ECD10436F4E786
:1007E000564B002688F800605E602C4600F02AFB1D
:1007F0001DB1002C18BF4FF00009FFF7F1FD63E7B2
:10080000002D3FF476AF002C3FF473AF022088F840
:10081000000000F0D3FA322000F0BAF9B0F1000A7B
:10082000C0F279811AF0030540F07581DBF80820E9
:1008300006EB0A03934200F26E81BAF5807F00F264
:100840006A81444B019355450DDA4FF47A7000F0FC
:100850009FF90290029A002AC0F25D81019B029AE0
:10086000EA540135EEE7C820FFF7B2FD054600283F
:1008700000F051811F2E11D8C6F12004544528BF25
:1008800054460EAB26F0030022463249184400F0CD
:10089000A7FA2246FF212F4800F0CCFA4FEAAA0A15
:1008A0005FFA8AF22B493046FFF7B8FD044600286C
:1008B00081D006EB8A06054698E70220FFF788FDFF
:1008C00000283FF416AFFFF799FD00283FF411AF61
:1008D00000229246DBF808309A4259D21F2A1ED8CD
:1008E0000E9B01331BD022F0030316A90B4453F8CF
:1008F000203C09931848436883B3174800210DF141
:10090000240E11F80E3083EA0A03DBB2013150F8ED
:100910002330042983EA1A2AF3D10432DAE7104695
:10092000019200F0B1F9019A0990E3E75024012007
:100930009C2501205C240120B5040008A029012089
:10094000982401207E3400085424012058240120DA
:10095000803400089C240120A025012019464FF076
:10096000080E11F0010F4FEA51011FBF81F06D41D8
:1009700081F4380181F4034181F02001BEF1010EC0
:10098000EFD140F823100133B3F5807FE6D1B4E70F
:1009900016A8042140F84CAD00F048F926E716A847
:1009A000002340F8343D642100F01CF900287FF456
:1009B000A0AE0220FFF70CFD00283FF49AAE099884
:1009C00000F092F916AB43F8480D04211846E3E70E
:1009D00016A8002340F8343D642100F003F90028F4
:1009E0007FF487AE0220FFF7F3FC00283FF481AECE
:1009F000099800F087F916AB43F8440DE5E70220AB
:100A0000FFF7E6FC00283FF474AE00F081F916AB66
:100A100043F8400DD9E70220FFF7DAFC00283FF445
:100A200068AE09A9142000F079F9824616A80421BD
:100A300040F83CAD00F0FAF8514609A8ACE7322086
:100A400000F0A6F8B0F1000AFFF653AE1AF0030F5B
:100A50007FF44FAEDBF808200AEB070393423FF622
:100A600048AE0220FFF7B4FC00283FF442AE2AF063
:100A7000030ABA44BA453FF4B9AE384600F004F967
:100A80000421089008A800F0D1F80437F2E74FF4E9
:100A90007A70FFF79DFC00283FF42BAEFFF7AEFC09
:100AA00000283FF489AE0E9B01330CD008220EA91A
:100AB0000020FFF7B3FC00283FF47EAE2022FF2188
:100AC0000EA800F0B7F9FFF78BFC304800F038FFB4
:100AD00006E616A8002340F8343D642100F082F8B1
:100AE000824600287FF405AE0220FFF771FC002843
:100AF0003FF4FFADFFF774FC41F2883000F020FFB7
:100B0000099800F0D3F9D14600F09CF9DCE50546E0
:100B10006CE60027EDE52546EBE5002000F038F80F
:100B20000290029B002BFFF6D2AD012000F03CF9B1
:100B3000029B213B122B3FF6C7AD01A252F823F0D6
:100B4000E70600080507000873070008C906000843
:100B5000C9060008C9060008010800083F0A000885
:100B6000BB0800089F090008D1090008FF09000818
:100B7000C9060008170A0008C90600088F0A0008FD
:100B8000ED070008C9060008D30A0008A086010086
:100B900037B5114B1A780132D2B20024012A01462E
:100BA0008DF8074011D80D4803681D6A4FF47A7319
:100BB0004B4301220DF10701A847012805D1084B3D
:100BC0009DF807001C7003B030BD4FF4FA7000F0C0
:100BD000B7FE4FF0FF30F6E700240120F029012096
:100BE000AC29012038B50E4B1A780132D2B2012A55
:100BF00005460ED80B4803681C6A4FF47A734B43C2
:100C000004222946A047042803D1074B002018706E
:100C100038BD4FF4FA7000F093FE4FF0FF3038BD4E
:100C200000240120F0290120AC29012030B4054C1A
:100C30002368DD69044B0A46AC460146204630BCB9
:100C4000604700BFF0290120A0860100F8B501F03F
:100C5000ADF8094C094E0A4F207000253068237802
:100C6000834207D901F09CF8336805440133BD4243
:100C70003360F3D9F8BD00BFAD290120A8290120B8
:100C8000FF7F010001F050B900F1006000F5C030B5
:100C90000068704700F10060920000F5C03001F07C
:100CA000DBB80000054B1A68054B1B789B1A834282
:100CB00002D9104401F074B800207047A82901201F
:100CC000AD29012038B5074D04462868204401F0BD
:100CD0006FF828B928682044BDE8384001F080B892
:100CE00038BD00BFA829012010F0030308D1B0F5DA
:100CF000806F05D800F10050A0F5712000687047A2
:100D000000207047014BC058704700BF20F4F01F0F
:100D1000014B1868704700BF002004E0F0B5204B7D
:100D20001E68204B1F885D6893F90840C6F30B02CC
:100D3000BA424FEA164622D09F89BA4221D01F8B71
:100D4000BA4206D102220C2404FB02335D6893F9F7
:100D50000840B6F5805F16D041F201039E4208BFFD
:100D60005A24421E0A44013D0B46934215D215F9FE
:100D7000016F581C4EB1034600F8016CF5E70022E4
:100D8000E1E70122DFE74124EBE72C2582421D70D9
:100D900001D9981C5C70401AF0BD1846FBE700BFF3
:100DA000002004E004240120022802BF024B4FF47B
:100DB00080229A61704700BF00000240022802BFF3
:100DC000014B04229A61704700000240022801BFD3
:100DD000024A536983F004035361704700000240E4
:100DE00010B50023934203D0CC5CC4540133F9E71F
:100DF00010BD000030B5441E14F9010F0B4660B160
:100E000093F90050854201F1010106D11AB993F915
:100E10000020801A30BD013AEEE7002AF7D11046D3
:100E200030BD000002460346981A13F9011B002941
:100E3000FAD1704702440346934202D003F8011BE3
:100E4000FAE77047024B1A78024B1A70704700BFDE
:100E5000AC2901200024012038B5104D104C284643
:100E600000F0A8F82146284600F0D0F823680D4885
:100E7000DA6ED2F8043843F00203C2F8043800F006
:100E80005FFD0949206800F0D5F92368DA6ED2F8D1
:100E9000043823F00203C2F8043838BDF0290120D9
:100EA0002C35000840420F007835000870470000DC
:100EB00072B6202383F3118862B6704702684368D4
:100EC0001143016003B118477047000013B5446B2C
:100ED000D4F894341A681178042915D1217C022998
:100EE00012D11979128901238B4013420CD101A927
:100EF00004F14C0001F070FED4F89444019B217978
:100F00000246206800F0E6F902B010BD143001F08E
:100F1000F5BD00004FF0FF33143001F0EFBD0000CD
:100F20004C3001F0C5BE00004FF0FF334C3001F0F3
:100F3000BFBE0000143001F0C5BD00004FF0FF310E
:100F4000143001F0BFBD00004C3001F091BE000034
:100F50004FF0FF324C3001F08BBE0000D0F89424EB
:100F600038B5136819780429054601D0012038BD29
:100F7000017C0229FAD112795C8901209040044059
:100F8000F4D105F1140001F057FD02460028EDD020
:100F9000D5F894544FF480732868697900F088F983
:100FA000204638BD406BFFF7D9BF000000207047D6
:100FB000704700007FB5124B0360002343608360DD
:100FC000C360012502260F4B05740446029001936D
:100FD00000F18402294600964FF48073143001F02A
:100FE00007FD094B0193029400964FF4807304F5BA
:100FF0002372294604F14C0001F0CAFD04B070BD13
:10100000B0340008A50F0008CD0E000808B50A6826
:10101000FFF74EFF0B7902EB830318624B790D3318
:1010200042F823008B7913B102EB83021062022392
:101030000374C0F89414002383F3118808BD0000E2
:1010400038B5037F044613B190F85430ABB9201D76
:1010500001250221FFF732FF04F1140025776FF01C
:10106000010100F095FC84F8545004F14C006FF03D
:101070000101BDE8384000F08BBC38BD10B501213E
:1010800004460430FFF71AFF0023237784F8543016
:1010900010BD000038B504460025143001F0C0FC36
:1010A00004F14C00257701F08BFD201D84F854508D
:1010B0000121FFF703FF2046BDE83840FFF74EBF90
:1010C00090F85C3003F06003202B19D190F85D207C
:1010D000212A0AD0222A4FF000030ED0202A0FD155
:1010E000084A02650722426504E0064B03650723B0
:1010F0004365002383650120704703654365F9E775
:101100000020704728240120D0F8943437B51A689D
:101110001178042904461AD1017C022917D11979C2
:10112000128901238B40134211D100F14C0528464E
:1011300001F004FE58B101A9284601F04DFDD4F894
:101140009444019B21790246206800F0C3F803B063
:1011500030BD000000EB8103F7B51C6A05460E4662
:10116000ECB105EB8607FFF7A3FE201D0821FFF772
:10117000A5FEFB685B691B684C3413B1204601F087
:1011800039FD01A9204601F027FD024648B1019B27
:101190003146284600F09EF8002383F3118803B0FF
:1011A000F0BDFB685A691268002AF5D01B8A013B22
:1011B0001340F1D105F15C02EAE700000D3138B5CA
:1011C00050F82140D4B1FFF773FED4F8942413688B
:1011D000527903EB8203DB689B695D6845B10421AA
:1011E0006018FFF76BFE294604F1140001F02EFC95
:1011F0002046FFF7B3FE002383F3118838BD0000BB
:101200007047000072B6202383F3118862B67047DE
:1012100000F0B4BF012303700023436000F12402F7
:1012200000F1380142F8043B8A421361FAD103818C
:101230004381704738B50446FFF7E4FF002541605D
:10124000C560056145618561C561056200F0A6FF65
:101250000223237085F3118838BD000070B500EBC0
:10126000810305465069DA600E46144618B1102213
:101270000021FFF7DFFDA06918B110220021FFF760
:10128000D9FD31462846BDE8704001F051B8000054
:10129000028902F001020281428902F001024281C8
:1012A0000022026142618261C261026201F0D4B82F
:1012B000F0B400EB81044789E4680125A4698D40FE
:1012C0003D43458123600023A2606360F0BC01F0D0
:1012D000EFB80000F0B400EB81040789E468012551
:1012E00064698D403D43058123600023A2606360F3
:1012F000F0BC01F06BB9000070B502230025044674
:101300000370A0F8645080F8665080F8675005813B
:101310004581C560056145618561C561056280F8EB
:101320004C5000F0A1FF63681B6823B1294620469A
:10133000BDE87040184770BD436802781B6880F8AC
:101340006820052202700BB1042118477047000085
:10135000436890F868201B6802700BB1052118479C
:101360007047000090F84C3070B5044613B100236C
:1013700080F84C3004F15C02204601F08FF863687D
:101380009B6863BB94F85C5015F0600615D194F827
:101390005D3005F07F0545EA032540F202339D42AA
:1013A00000F00B8159D8022D00F0D9803DD8002DD6
:1013B00000F08580012D00F0CC800021204601F056
:1013C000DDFA0021204601F0CFFA63681B6813B1F3
:1013D000062120469847062384F84C3070BD2046ED
:1013E00098470028CED094F8632094F8623043EAFE
:1013F0000223626D934238BF636594F95C30656D7A
:10140000002B80F2FC80002D00F0EB80092384F893
:101410004C30FFF7F7FE636D226D00212046FFF789
:1014200059FF002383F3118870BDB5F5817F00F06B
:10143000B080B5F5407F49D0B5F5807FBDD194F837
:101440005E30012BB9D1B4F8643023F00203A4F864
:10145000643026656665A665C5E740F201639D4276
:101460001ED8B5F5C06F3BD2B5F5A06FA5D1B4F8C5
:101470005C30B3F5A06F0ED194F85E3084F866301E
:10148000204600F049FF63681B6813B10121204624
:10149000984703232370002323656365A365A2E7B0
:1014A000B5F5106F32D040F602439D4251D0B5F5EC
:1014B000006F82D104F167032365012324E004F166
:1014C0006403236502236365A5658CE794F85E30A9
:1014D000012B7FF472AFB4F8643043F00203B6E737
:1014E00094F86120616894F860304D6894F85F105A
:1014F00043EA0223204694F85E20A84700283FF4E0
:101500005CAF4368236503686365A4E72378042B15
:101510000FD1FFF777FE2046FFF7BAFE86F311885A
:10152000636884F867601B68032121700BB1204653
:10153000984794F85E30002BADD084F867300423D0
:10154000237063681B68002BA5D0022120469847B2
:10155000A1E7374B23650223636500239EE794F8D8
:10156000601011F0800F204601F00F010ED000F046
:1015700087FF012806D002287FF41FAF2D4B23657B
:10158000606568E72C4B2365656564E700F06AFFDA
:10159000EFE794F85E30002B7FF40FAF94F86030E3
:1015A00013F00F013FF477AF1A06204602D501F081
:1015B000F9F970E701F0ECF96DE794F85E30002B73
:1015C0007FF4FBAE94F8603013F00F013FF463AF8B
:1015D0001B06204602D501F0D1F95CE701F0C4F901
:1015E00059E7142384F84C30FFF70CFE2B462A46AB
:1015F00029462046FFF75CFE85F3118870BD5DB17A
:10160000152384F84C30FFF7FDFD636D226D00213A
:101610002046FFF74DFE04E70B2384F84C30FFF71C
:10162000F1FD2B462A4629462046FFF753FEE3E705
:10163000E0340008D8340008DC34000838B590F8ED
:101640004C300446152B28D8DFE803F03C27272729
:1016500027273C27270B2837272727272727272710
:101660003C3C90F8631090F86220436D42EA0122FE
:101670009A4213D9C268128AB3FBF2F502FB153500
:1016800065B9FFF7BFFD2B462A462946FFF722FE24
:1016900085F311880A2384F84C3038BD142384F86C
:1016A0004C30FFF7AFFD00231A4619462046FFF7DE
:1016B000FFFD002383F3118838BD836D03B1984784
:1016C0000023E8E7002101F059F90021204601F04C
:1016D0004BF963681B6813B106212046984706231F
:1016E000D9E7000090F84C20152A38B5044621D8D7
:1016F0000123934040F6416213421CD113F480153C
:101700000ED19B0216D50B2380F84C30FFF77AFDE3
:101710002B462A462946FFF7DDFD85F3118838BDA3
:10172000C3689B695B682BB9836D03B1984700233D
:1017300084F84C3038BD002101F020F9002120460A
:1017400001F012F963681B6813B10621204698471F
:101750000623EDE7024B00221B605B609A60704736
:10176000B0290120002303748268054B1B68996827
:101770009142FBD25A680360426010605860704723
:10178000B029012008B572B6202383F3118862B610
:10179000037C032B05D0042B0DD02BB983F31188C8
:1017A00008BD436900221A604FF0FF334361FFF721
:1017B000D9FF0023F2E790E80C001A60026853603A
:1017C000F2E70000002303748268054B1B689968E8
:1017D0009142FBD85A6803604260106058607047BD
:1017E000B0290120054B19690874186802681A604D
:1017F0005360186101230374FEF796BDB0290120E0
:1018000030B54B1C87B005460A4C10D023690A4AF4
:1018100001A800F0D9F82846FFF7E4FF049B13B1B4
:1018200001A800F00DF92369586907B030BDFFF732
:10183000D9FFF8E7B02901208517000838B50C4D0D
:1018400041612B6981689A689142044603D8BDE8DA
:101850003840FFF787BF1846FFF784FF01232C614C
:10186000014623742046BDE83840FEF75DBD00BF49
:10187000B0290120044B1A681B6990689B68984244
:1018800094BF002001207047B029012010B5084CFA
:10189000236820691A6822605460012223611A7447
:1018A000FFF790FF01462069BDE81040FEF73CBD00
:1018B000B029012072B6202383F3118862B67047E5
:1018C0008260022202740022427470478368A3F18E
:1018D0007C0243F80C2C026943F83C2C426943F823
:1018E000382C074A43F81C2CC26843F8102C0222FB
:1018F00003F8082C002203F8072CA3F11800704706
:101900004103000810B5FFF7D5FFFFF7DFFF002107
:101910000446FFF793FF002383F31188204610BD90
:10192000024B1B6958610F20FFF75CBFB0290120F3
:1019300008B5FFF7BFFFBDE80840FFF7F1BF0000A3
:1019400008B50146FFF7B6FF0820FFF759FF00234F
:1019500083F3118808BD000049B1064B42681B693A
:1019600018605A60136043600420FFF749BF4FF0CE
:10197000FF307047B02901200368984206D01A68EA
:101980000260506059611846FFF7ECBE70470000D6
:1019900038B504460D462068844200D138BD03683E
:1019A00023605C604561FFF7DDFEF4E7054B03F162
:1019B00014025A619A614FF0FF32DA6100221A6212
:1019C000704700BFB0290120F8B503614FF0804394
:1019D000C2605C6A194B1A46022952F8145F38BF7C
:1019E0000221954206461F460AD1586198611C6241
:1019F0000560456081600819BDE8F84001F0C0B994
:101A0000186AAB68241A0C1902D3E41A2D6804E092
:101A10009C4202D2204401F0C1F9AB689C42F4D848
:101A20006B68736035601E606E60B460A9684FF0CB
:101A3000FF33091BA960FB61F8BD00BFB02901207D
:101A400010B41B4C234653F8141F814210D0416838
:101A500002680A60026851609A424FF00001C1605A
:101A600003D0936881680B4493605DF8044B704722
:101A70000A68626100209A425360C86003D15DF831
:101A8000044B01F085B993688868034493604FF074
:101A90008042206A526A121A9342E6D9991A0129A1
:101AA00098BF931C18445DF8044B01F077B900BF50
:101AB000B029012000207047FEE7000070470000B9
:101AC0004FF0FF307047000072B6202383F3118877
:101AD00062B67047022906D0032906D001290648BC
:101AE00018BF0020704705487047032A9ABF044872
:101AF00000EBC20000207047D4350008883500088C
:101B00003024012070B5044608460D46FFF78AF9D7
:101B1000C6B22046013403780BB9184670BD324670
:101B20002946FFF767F90028F3D1012070BD0000B6
:101B30002DE9F04F80469BB008460C461646FFF74D
:101B400071F93A49C5B22046FFF7DCFF08B101350B
:101B5000EDB237492046FFF7D5FF08B11035EDB299
:101B6000632D01AF0CD8DFF8D490DFF8D4A03D4648
:101B700094F800B0BBF1000F1CD185F800B003E071
:101B80002146384601F072FC3846FFF74BF9C0B2E7
:101B9000431C5B0088E84800337003237370002304
:101BA00002361946DAB2904206F1020636D81BB068
:101BB000BDE8F08FBBF1250F2BD107221B49204632
:101BC000FFF718F940B9DAF800302B60DAF8043082
:101BD0006B6007340835CBE7082215492046FFF72C
:101BE00009F9B0B91349AB1C11F8012F100902F023
:101BF0000F0210F8090012F8092003F8012C0E4A10
:101C000003F8020C914203F10203EDD118350834B8
:101C1000AEE785F800B001340135A9E7FA5C06F8B3
:101C2000022C06F8011C0133BCE700BF3435000864
:101C30003C3500081FF4F01F2BF4F01F4E35000850
:101C40004535000808B5FFF73FFF0348FFF75CFA8A
:101C5000002383F3118808BDF029012010B5044644
:101C6000052915D8DFE801F015140315151BFFF73A
:101C70002BFF0E4A0121FFF7F1FA20460C4A022100
:101C8000FFF7ECFA0B48FFF705FA002383F31188FE
:101C900010BDFFF719FF0748FFF7D2F9F5E7FFF787
:101CA00013FF0448FFF7EAF9EFE700BFE434000848
:101CB00008350008F029012038B50C4D0C4C0D49B1
:101CC0002A4604F10800FFF733FF05F1CA0204F1C8
:101CD00010000949FFF72CFF05F5CA7204F118003E
:101CE0000649BDE83840FFF723BF00BFB82E0120EA
:101CF00030240120603500086A3500083C350008B2
:101D0000BFF34F8F024AD368DB03FCD4704700BF98
:101D1000003C024008B5074B1B7853B9FFF7F0FFB2
:101D2000054B1A69002ABFBF044A5A6002F1883283
:101D30005A6008BD16310120003C0240230167456E
:101D400008B5054B1B7833B9FFF7DAFF034A13696F
:101D500043F00043136108BD16310120003C0240EE
:101D6000072870B513D80B4A0B4C137863B90B4E88
:101D70004FF0006144F8231056F823500133082B2C
:101D80002944F7D10123137054F8200070BD0020BE
:101D900070BD00BF3831012018310120F435000832
:101DA000014B53F820007047F435000808207047B5
:101DB000072810B5044601D9002010BDFFF7D0FF59
:101DC000064B53F824301844C21A0BB9012010BD39
:101DD00012680132F0D1043BF6E700BFF435000889
:101DE000072810B504462FD8FFF78AFFFFF792FFA8
:101DF0001649F323CB60FFF783FFC300DBB243F444
:101E0000007343F002030B610B6943F480330B61F1
:101E1000FFF776FFFFF7A4FF0D4B53F82430034480
:101E2000BFF34F8F0B4A98420AD3BFF34F8FBFF3D4
:101E30006F8FFFF785FF2046BDE81040FFF7B8BF62
:101E4000C2F85C022030EEE7002010BD003C0240EA
:101E5000F435000800ED00E02DE9F84312F001032D
:101E6000154643D10244B2F1016F3FD22C4B1B689F
:101E700013F001033AD02B4CFFF74CFFF323E36040
:101E8000FFF73EFF40F20127032D16D8254C0F46E1
:101E9000401A40F20118EB1B0B44012B00EB070624
:101EA000236926D823F001032361FFF749FF0120AE
:101EB000BDE8F883043D0430E6E78307E6D12369F3
:101EC00023F44073236123693B43236151F8046B7E
:101ED0000660BFF34F8FFFF713FF03689E42E9D000
:101EE000236923F001032361FFF72AFF0020BDE8E7
:101EF000F88323F440732361236943EA08032361D1
:101F0000B94637F8023B3380BFF34F8FFFF7F8FE37
:101F10003688B9F80030B6B2B342BCD0E0E700BFB3
:101F200000380240003C0240084908B50B7828B14F
:101F300053B9FFF7EFFE01230B7008BD23B1BDE8D5
:101F400008400870FFF7FCBE08BD00BF1631012035
:101F5000014B53F820007047502800400A4B1A6F7D
:101F6000120407D41A6F42F400721A671A6F42F40F
:101F700000421A67054A136843F48073136000B285
:101F8000034B43F8201070470038024000700040B7
:101F900050280040014B1868704700BF502800408F
:101FA00001460020FFF7DABF38B5094B1B689B00DC
:101FB0000CD5084B084D01221A700024E0B2FFF73F
:101FC000C7FF45F824000134082CF7D138BD00BF05
:101FD000743802405C3101203C310120014B1878FB
:101FE000704700BF5C310120F0B5BFF34F8FBFF3E6
:101FF0006F8F1D4B0021C3F85012BFF34F8FBFF3FB
:102000006F8F5A6942F400325A61BFF34F8FBFF3AA
:102010006F8FC3F88410BFF34F8FD3F88020C2F3C3
:10202000C904C2F34E325201A50743F6E07602EA34
:10203000060E284621464EEA00070139C3F86072B1
:102040004F1C00F14040F6D1203A12F1200FEED1A2
:10205000BFF34F8F5A6942F480325A61BFF34F8FFA
:10206000BFF36F8FF0BD00BF00ED00E0FEE70000A2
:10207000084A094B09498B4204D3094A002193427B
:1020800005D3704752F8040F43F8040BF3E743F805
:10209000041BF4E7EC3700086834012068340120A1
:1020A00068340120036F30B500229D68C46E11466C
:1020B0004FF0FF3004EB421301329542C3F8001990
:1020C000C3F81019C3F80809C3F8001BC3F8101BA4
:1020D000C3F8080BEED24FF00113C4F81C3830BD22
:1020E000890141F02001016103699B06FCD41220A3
:1020F00000F0E4BE204B03EB80022DE9F047D2F85C
:102100000CE0DD6EDEF81420461CD2F800C005EBB2
:10211000063605EB4018516861450BD3D5F83428D5
:10212000012303FA00F022EA0000C5F8340818463B
:10213000BDE8F087BEF81040ACEB0103A34228BF16
:102140002346D8F81849A4B2B3EB840F10D894688A
:102150001F46A4F1040959F804AFC6F800A0042FE3
:1021600001D9043FF7E71C440B4494605360D2E765
:102170000020BDE8F08700BF6031012010B5054C9C
:102180002046FFF747F84FF0A043E366024B236772
:1021900010BD00BF60310120383600080378012BE4
:1021A00070B5054650D12A4BC46E98421BD1294BBD
:1021B0005A6B42F080025A635A6D42F080025A65AF
:1021C0005A6D5A6942F080025A615A6922F08002BF
:1021D0005A610E2143205B6900F0EEFB1E4BE36069
:1021E0001E4BC4F800380023C4F8003EC02323600F
:1021F000EE6E4FF40413A3633369002BFCDA012362
:1022000033610C2000F05AFE3369DB07FCD4122046
:1022100000F054FE3369002BFCDA0026A660284645
:10222000FFF740FF6B68C4F81068DB68C4F81468F7
:10223000C4F81C684BB90A4BA3614FF0FF336361CC
:10224000A36843F00103A36070BD064BF4E700BF31
:102250006031012000380240401400400300200299
:10226000003C30C0083C30C0F8B5C46E05460021C3
:102270002046FFF735FF296F00234FF001128F68CA
:10228000C4F834384FF00066C4F81C284FF0FF3013
:1022900004EB431201339F42C2F80069C2F8006B9D
:1022A000C2F80809C2F8080BF2D20B68EA6E6B6735
:1022B000636210231361166916F01006FBD1122019
:1022C00000F0FCFDD4F8003823F4FE63C4F80038B5
:1022D000A36943F4402343F01003A3610923C4F826
:1022E0001038C4F814380A4BEB604FF0C043C4F800
:1022F000103B084BC4F8003BC4F81069C4F800391F
:102300006B6F03F1100243F480136A67A362F8BD98
:102310001436000840800010C26E90F86610D2F8A3
:10232000003823F4FE6343EA0113C2F80038704713
:102330002DE9F0410EB200EB86080D46D8F80C10DE
:102340000F6807F00303022B50D0032B50D03D4AF7
:102350003D4F012B18BF1746C46E4FEA451E04EBD4
:102360000E030022C3F8102B8A6905F1100C002A15
:1023700040D04A8A05F158035B013A43E2500123F9
:10238000D4F81C2803FA0CF31343A6444A69C4F892
:102390001C380023CEF8103905F13F03002A39D04C
:1023A0000A8A898B9208012988BF4A43416F04EB4E
:1023B0008303561841EA0242466729465A6020467E
:1023C000FFF78EFED8F80C301B8A43EA85531F4373
:1023D00005F148035B01E7500123D4F81C2803FAF8
:1023E00005F51543C4F81C58BDE8F081174FB3E755
:1023F000174FB1E704EB4613D3F8002B22F4004249
:10240000C3F8002BD4F81C28012303FA0CF322EAAA
:102410000303BAE704EB83030E4A5A6004EB461643
:1024200029462046FFF75CFED6F8003923F4004326
:10243000C6F80039D4F81C38012202FA05F523EA5F
:102440000505CFE700800010008004100080081010
:1024500000800C1000040002026F12684267FFF750
:1024600021BE00005831C36E49015B5813F400408F
:1024700004D013F4001F14BF012002207047000095
:102480004831C36E49015B5813F4004004D013F483
:10249000001F14BF012002207047000000EB8101E3
:1024A000CB68196A0B6813604B6853607047000073
:1024B00000EB810330B5DD68AA691368D36019B9F0
:1024C000402B84BF402313606B8A1468C26E1C4487
:1024D000013CB4FBF3F46343033323F0030302EB47
:1024E000411043EAC44343F0C043C0F8103B2B689B
:1024F00003F00303012B09B20ED1D2F8083802EB26
:10250000411013F4807FD0F8003B14BF43F0805398
:1025100043F00053C0F8003B02EB4112D2F8003BFD
:1025200043F00443C2F8003B30BD00002DE9F04108
:10253000254DEE6E06EB40130446D3F8087BC3F836
:10254000087B38070AD5D6F81438190706D505EBE5
:1025500084032146DB6828465B689847FA0731D533
:10256000D6F81438DB072DD505EB8403D968DCB920
:102570008B69488A5E68B6FBF0F200FB12629AB97A
:102580001868DA6890420FD2121A83E8140072B603
:10259000202383F3118862B60B482146FFF788FF9A
:1025A00084F31188BDE8F081012303FA04F26B89FA
:1025B00023EA02036B81CB6823B121460248BDE8C0
:1025C000F0411847BDE8F0816031012000EB810344
:1025D00070B5DD68C36E6C692668E6604A0156BB5B
:1025E0001A444FF40020C2F810092A6802F00302CE
:1025F000012A0AB20ED1D3F8080803EB421410F4F2
:10260000807FD4F8000914BF40F0805040F00050A3
:10261000C4F8000903EB4212D2F8000940F004406C
:10262000C2F80009D3F83408012202FA01F101438B
:10263000C3F8341870BD19B9402E84BF4020206003
:1026400020682E8A841940F00050013C1A44B4FBE3
:10265000F6F440EAC440C6E7F8B504461F48C56E24
:1026600005EB4413D3F80869C3F80869F10719D5D5
:10267000D5F81038DA0715D500EB8403D9684B6913
:102680001F68DA6897421AD2D21B00271A605F606F
:1026900072B6202383F3118862B62146FFF796FFB6
:1026A00087F31188330617D5D5F834280123A340C2
:1026B000134211D02046BDE8F840FFF71BBD0123AF
:1026C00003FA04F2038923EA020303818B68002BD7
:1026D000E8D021469847E5E7F8BD00BF603101200A
:1026E000A0482DE9F84FC56E6E69AB691E4016F41F
:1026F000805F6E61044605D0FEF7FEFDBDE8F84F31
:1027000000F07EBC002E12DAD5F8003E95489B07FB
:102710001EBFD5F8003E23F00303C5F8003ED5F8F0
:10272000043823F00103C5F80438FEF711FE37051D
:1027300002D58C48FEF700FEB0040CD5D5F8083859
:1027400013F0060FEB6823F470530CBF43F41053DF
:1027500043F4A053EB60310704D56368DB680BB129
:1027600080489847F2026FD4B3020CD5D4F86C803D
:10277000DFF8F0A100274FF00109236F9B68F9B241
:102780008B4280F09C80F70619D5E16E0A6AC2F38D
:102790000A1702F00F0302F4F012B2F5802F00F0D6
:1027A000B680B2F5402F0AD104EB830301F58051C6
:1027B000DB68186A00231A469F4240F09C8033036E
:1027C000D5F818481DD5E70302D50020FFF7AEFE67
:1027D000A50302D50120FFF7A9FE600302D5022060
:1027E000FFF7A4FE210302D50320FFF79FFEE202BC
:1027F00002D50420FFF79AFEA30202D50520FFF7B9
:1028000095FE77037FF57AAFE60702D50020FFF744
:1028100023FFA50702D50120FFF71EFF600702D5A1
:102820000220FFF719FF210702D50320FFF714FF4D
:10283000E20602D50420FFF70FFFA3067FF55EAF87
:102840000520FFF709FF59E7D4F86C80DFF814A1E1
:1028500000274FF00109236F9B685FFA87FB5B45F8
:1028600082D308EB4B13D3F8002902F44022B2F5CF
:10287000802F22D1D3F80029002A1EDAD3F80029AC
:1028800042F09042C3F80029D3F80029002AFBDB6C
:102890005946E06EFFF724FC228909FA0BF322EA7D
:1028A0000303238104EB8B03DB689B6813B1594658
:1028B000504698475846FFF71DFC0137CBE708EB19
:1028C0004112D2F8003B03F44023B3F5802F10D11E
:1028D000D2F8003B002B0CDA628909FA01F322EAF4
:1028E0000303638104EB8103DB68DB680BB15046B3
:1028F0009847013741E79C0708BF0A68072B98BF34
:10290000027003F101039CBF120A013054E7023345
:1029100004EB830201F58051526890690268D0F897
:1029200008C04068A2EB000E0022104697420AD170
:1029300004EB830463689B699A683A449A605A6816
:1029400017445F603BE712F0030F08BF0868964525
:1029500088BF8CF8000002F1010284BF000A0CF16C
:10296000010CE3E760310120C36E03EB4111D1F8A4
:10297000003B43F40013C1F8003B7047C36E03EB08
:102980004111D1F8003943F40013C1F80039704700
:10299000C36E03EB4111D1F8003B23F40013C1F8DF
:1029A000003B7047C36E03EB4111D1F8003923F4AB
:1029B0000013C1F80039704700F1604300F01F02B6
:1029C000400903F5614309018000C9B200F160408C
:1029D00083F8001300F5614001239340C0F8803173
:1029E0000360704772B6202383F3118862B6704784
:1029F00030B5039C0172043304FB0325C361049BBF
:102A000003630021059B00604060C1604261026178
:102A10008561046242628162C162436330BD00002D
:102A20000022416A41610161C2608262C2626FF04C
:102A30000101FEF7ADBF000003694269934203D173
:102A4000C2680AB100207047181D704703691960F9
:102A5000C2680132C260C269134482690361934251
:102A600024BF436A03610021FEF786BF38B50446E0
:102A70000D46E3683BB16269131D1268A3621344FB
:102A8000E362002038BD237A33B929462046FEF799
:102A900063FF0028EDDA38BD6FF00100FBE70000AE
:102AA000C368C269013BC3604369134482694361DF
:102AB000934224BF436A436100238362036B03B1E3
:102AC0001847704770B50446FFF78CFF866A3EB919
:102AD000FFF7CCFF054618B186F31188284670BD74
:102AE000A36AE26A13F8015BA362934202D3204611
:102AF000FFF7D6FF002383F31188EFE72DE9F047B6
:102B000004460E4617469846FFF76CFF0025A94677
:102B1000D4F828A0BAF1000F09D141462046FFF7AA
:102B2000A5FF20B18AF311882846BDE8F087A16A85
:102B3000E36AA7EB050A5B1A9A4528BF9A46BAF1E1
:102B4000400F1BD9334601F1400251F8040B43F802
:102B5000040B9142F9D1A36A40334036A362403559
:102B6000A26AE36A9A4202D32046FFF799FF89F3EB
:102B70001188BD42D8D2FFF735FFC9E7304652462B
:102B8000FEF72EF9A36A53445644A3625544E7E77F
:102B900010B5029C0172043303FB0421C3610023BE
:102BA0008362C362039B0363049B00604060C46054
:102BB00042610261816104624262436310BD0000B0
:102BC000026AC260426A4261026100228262C2629B
:102BD0006FF00101FEF7DCBE436902699A4203D13E
:102BE000C2680AB100207047184650F8043B0B60D9
:102BF00070470000C368C2690133C360436913446E
:102C000082694361934224BF436A43610021FEF716
:102C1000B3BE000038B504460D46E3683BB12369F6
:102C20001A1DA262E2691344E362002038BD237AD0
:102C300033B929462046FEF78FFE0028EDDA38BD6D
:102C40006FF00100FBE7000003691960C268013AF8
:102C5000C260C269134482690361934224BF436A1C
:102C6000036100238362036B03B1184770470000C0
:102C700070B504460E46FFF7B5FE856A35B91146B4
:102C8000FFF7C8FF10B185F3118870BDA36A1E70ED
:102C9000A36AE26A01339342A36204D3E169204646
:102CA0000439FFF7D1FF002080F3118870BD0000C8
:102CB0002DE9F04704460D4690469946FFF792FEEF
:102CC0000026B246A76A4FB949462046FFF7A2FF41
:102CD00020B187F311883046BDE8F087A06AE76A23
:102CE000A8EB06033F1A9F4228BF1F46402F1BD95F
:102CF00005F1400355F8042B40F8042B9D42F9D10F
:102D0000A36A4033A3624036A26AE36A9A4204D3BC
:102D1000E16920460439FFF797FF8AF31188464599
:102D2000D9D2FFF75FFECDE729463A46FEF758F8BD
:102D3000A36A3B443D44A3623E44E5E7026943691C
:102D40009A4203D1C3681BB9184670470023FBE7BA
:102D5000836A002BF8D0043B9B1AF5D01360C3683C
:102D6000013BC360C3691A44836902619A4224BF6C
:102D7000436A0361002383620123E5E700F086B91B
:102D80004FF08043002258631A610222DA607047D4
:102D90004FF080430022DA60704700004FF080431C
:102DA00058637047FEE7000010B5194CFEF7D2FCDF
:102DB000FEF7FCFD802217492046FEF781FD012326
:102DC00044F8180C0374144B144AD96821F4E061D8
:102DD0000904090C0A431249DA60CA6842F0807299
:102DE000CA60104A1049C2F8B01F116841F00101D1
:102DF00011601022DA77202283F82220002383F347
:102E0000118862B60948BDE81040FEF77BBD00BFDF
:102E1000D82901204436000800ED00E00003FA053F
:102E2000F0ED00E0001000E055CEACC54C360008D7
:102E30002DE9F84F204C4FF00008656904F11407A4
:102E4000C1464FF08043266A5B6AAA689E1B964281
:102E50001FD34FF0200AAA68236AD5F80CB0134498
:102E600023622B68BB425F60A6EB02066361C5F874
:102E70000C8001D1FFF78CFF89F311882869D847AE
:102E800072B68AF3118862B66569AB689E42E2D277
:102E9000D7E76269BA420CD0916823628E1B9660B4
:102EA000A86802282CBF1818981CBDE8F84FFFF737
:102EB00075BFBDE8F88F00BFB0290120034B5968EA
:102EC0005A68521A9042FBD8704700BF001000E0C9
:102ED0004B6843608B688360CB68C3600B69436158
:102EE0004B6903628B6943620B68036070470000A3
:102EF00008B5274B27481A6940F2FF710A431A6147
:102F00001A6922F4FF6222F007021A611A691A6B29
:102F10000A431A631A6D0A431A651F4A1B6D11464C
:102F2000FFF7D6FF1D4802F11C01FFF7D1FF1C4837
:102F300002F13801FFF7CCFF1A4802F15401FFF704
:102F4000C7FF194802F17001FFF7C2FF174802F1ED
:102F50008C01FFF7BDFF164802F1A801FFF7B8FF8B
:102F6000144802F1C401FFF7B3FF134802F1E00176
:102F7000FFF7AEFF114802F1FC01FFF7A9FF10486F
:102F800002F58C71FFF7A4FFBDE8084000F0E0B83F
:102F900000380240000002406C3600080004024085
:102FA00000080240000C02400010024000140240E1
:102FB00000180240001C0240002002400024024091
:102FC0000028024008B500F035FAFFF7EDFEFEF7E5
:102FD000EBFFBDE80840FEF76FBE00007047000041
:102FE000064A536823F001035360EFF30983683303
:102FF00083F30988002383F31188704730EF00E0E2
:1030000010B572B6202383F3118862B6104B5B684B
:1030100013F4006318D0F1EE103AEFF309844FF087
:10302000807344F84C3C0B4BDB6844F8083CA4F13B
:10303000680383F30988FEF71DFC18B1064B44F8BA
:10304000503C10BD054BFAE783F3118810BD00BF5B
:1030500000ED00E030EF00E05103000854030008E9
:103060004FF0804310B51A6992070AD500241C61FD
:1030700072B6202383F3118862B6FFF7D9FE84F37A
:103080001188BDE81040FFF7BBBF0000104B1A6C61
:1030900042F001021A641A6E42F001021A660D4AE9
:1030A0001B6E936843F0010393604FF080436B22E3
:1030B0009A624FF0FF32DA6200229A615A63DA6054
:1030C0005A6001225A6108211A601C20FFF774BC63
:1030D00000380240002004E01B4B1A696FEA42529C
:1030E0006FEA52521A611A69C2F30A021A614FF06A
:1030F000FF301A695A69586100215A6959615A6941
:103100001A6A62F080521A621A6A02F080521A62D7
:103110001A6A5A6A58625A6A59625A6A0B4A10689D
:1031200040F480701060186F00F44070B0F5007FBC
:103130001EBF4FF4803018671967536823F400737B
:10314000536000F057B900BF0038024000700040E3
:10315000354B4FF080521A64344A4FF440411160AD
:103160001A6842F001021A601A689207FCD59A6840
:1031700022F003029A602C4B19469A6812F00C0256
:10318000FBD1186800F0F90018609A601A6842F4E0
:1031900080321A600B689B03FCD54B6F43F0010330
:1031A0004B67214B5A6F9007FCD5214A5A601A6829
:1031B00042F080721A601D4B1A4659684904FCD5CA
:1031C000196841F4803119605368D803FCD513683D
:1031D00043F400331360154A53689903FCD5124B2E
:1031E0001A689201FCD5134A9A6040F20112C3F8A2
:1031F0008C200022C3F890200F4A40F20731116062
:103200009A6842F002029A60074B9A6802F00C0238
:10321000082AFAD15A6C42F480425A645A6E42F437
:1032200080425A665B6E7047003802400070004072
:10323000086C400900948838003C0240084A08B5F0
:10324000536911680B4003F00103536123B1054A30
:1032500013680BB150689847BDE80840FFF7D0BE2F
:10326000003C0140E8330120084A08B55369116861
:103270000B4003F00203536123B1054A93680BB17D
:10328000D0689847BDE80840FFF7BABE003C01404F
:10329000E8330120084A08B5536911680B4003F070
:1032A0000403536123B1054A13690BB15069984770
:1032B000BDE80840FFF7A4BE003C0140E833012010
:1032C000084A08B5536911680B4003F008035361BD
:1032D00023B1054A93690BB1D0699847BDE808400E
:1032E000FFF78EBE003C0140E8330120084A08B5D4
:1032F000536911680B4003F01003536123B1054A71
:10330000136A0BB1506A9847BDE80840FFF778BED2
:10331000003C0140E8330120174B10B55C691A6886
:10332000144004F478725A61A30604D5134A936AD0
:103330000BB1D06A9847600604D5104A136B0BB1E5
:10334000506B9847210604D50C4A936B0BB1D06B98
:103350009847E20504D5094A136C0BB1506C9847A5
:10336000A30504D5054A936C0BB1D06C9847BDE812
:103370001040FFF745BE00BF003C0140E83301208C
:103380001A4B10B55C691A68144004F47C425A6107
:10339000620504D5164A136D0BB1506D984723058D
:1033A00004D5134A936D0BB1D06D9847E00404D552
:1033B0000F4A136E0BB1506E9847A10404D50C4A06
:1033C000936E0BB1D06E9847620404D5084A136F10
:1033D0000BB1506F9847230404D5054A936F0BB186
:1033E000D06F9847BDE81040FFF70ABE003C01408F
:1033F000E8330120062108B50846FFF7DDFA06216B
:103400000720FFF7D9FA06210820FFF7D5FA062191
:103410000920FFF7D1FA06210A20FFF7CDFA06218D
:103420001720FFF7C9FA06212820BDE80840FFF75A
:10343000C3BA000008B5FFF74FFE00F00BF8FDF728
:10344000E7FEFDF7B5FDFFF7C9FDBDE80840FFF752
:1034500095BC0000002304491A465A50C818083386
:10346000802B4260F9D17047E8330120034611F800
:10347000012B03F8012B002AF9D170471210121307
:103480001211000053544D3332463F3F3F3F3F3F00
:103490000053544D333246375B347C355D780053EE
:1034A000544D333246375B367C375D780000000080
:1034B00000000000290F0008150F0008510F000838
:1034C0003D0F0008490F0008350F0008210F0008C4
:1034D0000D0F0008AD0F0008000000000100000003
:1034E000000000000200000000000000551100086C
:1034F000BD11000840004000882E0120982E0120B8
:1035000002000000000000000300000000000000B6
:10351000011200080000000010000000A82E012089
:1035200000000000010000000000000060310120E8
:103530000101020025424F415244250025534552C6
:1035400049414C25004B616B75746546370030313D
:10355000323334353637383941424344454600002A
:103560004172647550696C6F740025424F4152443A
:10357000252D424C000000005D1C0008D51A0008F3
:10358000C1100008451C00084300000090350008E9
:1035900009024300020100C03209040000010202D6
:1035A0000100052400100105240100010424020289
:1035B0000524060001070582030800FF0904010035
:1035C000020A000000070501024000000705810211
:1035D0004000000012000000DC350008120110015C
:1035E0000200004083044057000201020301000072
:1035F0000403090400800000008000000080000037
:103600000080000000000200000004000000040030
:103610000000040000000000651300083D160008CB
:10362000E516000840004000D8310120D8310120C3
:1036300001000000E831012080000000400100008E
:10364000050000006D61696E00000000643600082E
:10365000F0310120E833012001000000A52D000811
:103660000000000069646C65000000001000802A02
:1036700000000000AAAAAAAA00000000FBFF0000A8
:103680000000000000A00A00000000000000000090
:10369000AAAAAAAA00000000FFFF00000000000084
:1036A000000000000000000000000000AAAAAAAA72
:1036B00000000000FFFF000000000000000000000C
:1036C0000000000000000000AAAAAAAA0000000052
:1036D000FFFF0000000000000000000000000000EC
:1036E00000000000AAAAAAAA00000000FFFF000034
:1036F00000000000000000000000000000000000CA
:10370000AAAAAAAA00000000FFFF00000000000013
:10371000000000000000000000000000AAAAAAAA01
:1037200000000000FFFF000000000000000000009B
:1037300000000000000000000A000000000000007F
:103740000300000000000000000000000000000076
:103750000000000000000000000000000000000069
:103760000000000000000000000000000000000059
:103770000000000000000000000000000000000049
:103780000000000000000000000000000000000039
:103790000000000000000000000000000000000029
:1037A000FF00000000000000843400083F0000001B
:1037B00049040000913400083F000000510400005B
:1037C0009F3400083F000000009600000000080041
:1037D00004000000F03500080000000000000000B8
:1037E00000000000000000000000000000000000D9
:00000001FF
